S1238000BD81B8CE827EBDFFCABDFFCDCE82A3BDFFCABD8222BD8222CE10001C0020BD82F5
S10C8020321D002020FE7EE00A5E
S123802AB680292621BD825ECC3E20FD1041CC2AB6FD1043C61EBD8222B61040B710405ACF
S123804A26F4BD80DF3B8101262CBD825ECC1C20FD1041CC1E9EFD1043BD8222BD8222BD83
S123806A8222BD81C8861EC601BD8222BD80FC4A26F5BD80DF3B8102262CBD825ECC1E2A01
S123808AFD1041CC2ACEFD1043BD8222BD8222BD8222BD81C8861EC602BD8222BD80FC4AF7
S12380AA26F5BD80DF3BBD825ECCCE3AFD1041CC1E00FD1043BD8222BD8222BD8222BD81E6
S12380CAC8861EC603BD8222BD80FC4A26F5BD80DF7F80293B36377C8029CC7A3AFD10417F
S12380EACC2A9EFD1043BD8222BD8222BD81C83332393CF71030F610302AFBF61031CE82D3
S123810A6E37545454543AE600F7104233C40FCE826E3AE600F710433839BD825ECE82CA9D
S123812ABDFFCABD8222BD8222BD8222CE82F1BDFFCACC7A60FD1041CCEEF6FD1043BD828E
S123814A22BD8222CC3A38FD1041CC1E00FD1043BD8222BD8222CCCE38FD1041CC1E00FDFF
S123816A1043BD8222BD8222CC1E9EFD1041CCB61EFD1043BD8222BD8222BD81C8BD81EB25
S123818ACC7A60FD1041CCEEF6FD1043BD8222BD8222CC7A3AFD1041CC2A9EFD1043BD822A
S12381AA22BD8222BD81C8BD8222BD82223BCE82F1BDFFCA7F8029BD81C8BD81D8397F1058
S12381CA407F10417F10427F10437F1044393637CC8124DDEFCC802ADDF20784AF0633323E
S12381EA393637C6098680BD8212BD825E44BD82225A26F38601C609BD8212BD825E48BDA7
S123820A82225A26F3333239B71040B71041B71042B71043B7104439183C18CE0003BD82B9
S123822A32180926F9183839183C18CEDF34180926FC1838393CCE10001D0010BD82511C29
S123824A0010BD82513839183C18CE0045180926FC183839183C18CE0096BD823F1809261F
S123826AF9183839FC60DAF266B6BEE0FEE6EE3E9C7A9E8E1B5B31323B3330484849542076
S123828A41204B455920544F20535441525420444941472054455354041B5B31323B333005
S12382AA4841435449564154494E4720494E46524152454420584D49545445522021200461
S12382CA1B5B31323B333048494E465241524544205349474E414C20444554454354454446
S10F82EA202020202020041B5B324A04CA
S9030000FC
